Microchip MPLAB XC8 Compiler V1.35 ()

Linker command line:

--edf=C:\Program Files\Microchip\xc8\v1.35\dat\en_msgs.txt -cs \
  -h+dist/default/production\OLED_Test.X.production.sym \
  --cmf=dist/default/production\OLED_Test.X.production.cmf -z -Q18F4550 \
  -oC:\Users\Brandy\AppData\Local\Temp\s66k.2 \
  -Mdist/default/production/OLED_Test.X.production.map -E1 -ver=XC8 \
  -ASTACK=060h-07ffh -pstack=STACK -ACODE=01000h-07FFFh \
  -ACONST=01000h-07FFFh -ASMALLCONST=01000h-010FFhx112 \
  -AMEDIUMCONST=01000h-07FFFh -ACOMRAM=01h-05Fh -AABS1=00h-07FFh \
  -ABIGRAM=01h-07FFh -ARAM=060h-0FFh,0100h-01FFhx7 -ABANK0=060h-0FFh \
  -ABANK1=0100h-01FFh -ABANK2=0200h-02FFh -ABANK3=0300h-03FFh \
  -ABANK4=0400h-04FFh -ABANK5=0500h-05FFh -ABANK6=0600h-06FFh \
  -ABANK7=0700h-07FFh -ASFR=0F60h-0FFFh \
  -preset_vec=01000h,intcode,intcodelo,powerup,init,end_init -pramtop=0800h \
  -psmallconst=SMALLCONST -pmediumconst=MEDIUMCONST -pconst=CONST \
  -AFARRAM=00h-00h -ACONFIG=0300000h-030000Dh -pconfig=CONFIG \
  -AIDLOC=0200000h-0200007h -pidloc=IDLOC -AEEDATA=0F00000h-0F000FFh \
  -peeprom_data=EEDATA \
  -prdata=COMRAM,nvrram=COMRAM,nvbit=COMRAM,rbss=COMRAM,rbit=COMRAM \
  -pfarbss=FARRAM,fardata=FARRAM,nvFARRAM=FARRAM \
  -pintsave_regs=BIGRAM,bigbss=BIGRAM,bigdata=BIGRAM -pbss=RAM \
  -pidata=CODE,irdata=CODE,ibigdata=CODE,ifardata=CODE -prparam=COMRAM \
  C:\Users\Brandy\AppData\Local\Temp\s66k.obj \
  dist/default/production\OLED_Test.X.production.obj 

Object code version is 3.11

Machine type is 18F4550

Call graph: (short form)




                Name                               Link     Load   Length Selector   Space Scale
C:\Users\Brandy\AppData\Local\Temp\s66k.obj
                end_init                           1000     1000        4      800       0
                idloc                            200000   200000        8   200000       0
                config                           300000   300000        E   300000       0
dist/default/production\OLED_Test.X.production.obj
                mediumconst                        6F4E     6F4E     10B2     37A7       0
                text23                             66EC     66EC       26     3376       0
                text22                             67BC     67BC       36     33DE       0
                text21                             690C     690C       84     3486       0
                text20                             67F2     67F2       40     33F9       0
                text19                             6660     6660        A     3330       0
                text18                             6674     6674       12     333A       0
                text17                             666A     666A        A     3335       0
                text16                             6654     6654        6     332A       0
                text15                             6686     6686       12     3343       0
                text14                             665A     665A        6     332D       0
                text13                             6738     6738       28     339C       0
                text12                             6990     6990       96     34C8       0
                text11                             6874     6874       46     343A       0
                text10                             66AA     66AA       16     3355       0
                text9                              66C0     66C0       16     3360       0
                text8                              6698     6698       12     334C       0
                text7                              6760     6760       2C     33B0       0
                text6                              6832     6832       42     3419       0
                text5                              68BA     68BA       52     345D       0
                text4                              6A26     6A26       A0     3513       0
                text3                              678C     678C       30     33C6       0
                text2                              6712     6712       26     3389       0
                text1                              6AC6     6AC6      106     3563       0
                text0                              6BCC     6BCC      382     35E6       0
                cstackCOMRAM                          1        1       29        1       1
                bssCOMRAM                            2A       2A        6        1       1
                cinit                              66D6     66D6       16     336B       0

TOTAL           Name                               Link     Load   Length     Space
        CLASS   STACK          

        CLASS   CODE           
                end_init                           1000     1000        4         0
                text23                             66EC     66EC       26         0
                text22                             67BC     67BC       36         0
                text21                             690C     690C       84         0
                text20                             67F2     67F2       40         0
                text19                             6660     6660        A         0
                text18                             6674     6674       12         0
                text17                             666A     666A        A         0
                text16                             6654     6654        6         0
                text15                             6686     6686       12         0
                text14                             665A     665A        6         0
                text13                             6738     6738       28         0
                text12                             6990     6990       96         0
                text11                             6874     6874       46         0
                text10                             66AA     66AA       16         0
                text9                              66C0     66C0       16         0
                text8                              6698     6698       12         0
                text7                              6760     6760       2C         0
                text6                              6832     6832       42         0
                text5                              68BA     68BA       52         0
                text4                              6A26     6A26       A0         0
                text3                              678C     678C       30         0
                text2                              6712     6712       26         0
                text1                              6AC6     6AC6      106         0
                text0                              6BCC     6BCC      382         0
                cinit                              66D6     66D6       16         0

        CLASS   CONST          

        CLASS   SMALLCONST     

        CLASS   MEDIUMCONST    
                mediumconst                        6F4E     6F4E     10B2         0

        CLASS   COMRAM         
                cstackCOMRAM                          1        1       29         1
                bssCOMRAM                            2A       2A        6         1

        CLASS   ABS1           

        CLASS   BIGRAM         

        CLASS   RAM            

        CLASS   BANK0          

        CLASS   BANK1          

        CLASS   BANK2          

        CLASS   BANK3          

        CLASS   BANK4          

        CLASS   BANK5          

        CLASS   BANK6          

        CLASS   BANK7          

        CLASS   SFR            

        CLASS   FARRAM         

        CLASS   CONFIG         
                config                           300000   300000        E         0

        CLASS   IDLOC          
                idloc                            200000   200000        8         0

        CLASS   EEDATA         



SEGMENTS        Name                           Load    Length   Top    Selector   Space  Class

                cstackCOMRAM                   000001  00002F  000030         1       1  COMRAM  
                reset_vec                      001000  000004  001004       800       0  CODE    
                text16                         006654  000006  00665A      332A       0  CODE    
                text14                         00665A  000006  006660      332D       0  CODE    
                text19                         006660  00000A  00666A      3330       0  CODE    
                text17                         00666A  00000A  006674      3335       0  CODE    
                text18                         006674  000012  006686      333A       0  CODE    
                text15                         006686  000012  006698      3343       0  CODE    
                text8                          006698  000012  0066AA      334C       0  CODE    
                text10                         0066AA  000016  0066C0      3355       0  CODE    
                text9                          0066C0  000016  0066D6      3360       0  CODE    
                cinit                          0066D6  000016  0066EC      336B       0  CODE    
                text23                         0066EC  000026  006712      3376       0  CODE    
                text2                          006712  000026  006738      3389       0  CODE    
                text13                         006738  000028  006760      339C       0  CODE    
                text7                          006760  00002C  00678C      33B0       0  CODE    
                text3                          00678C  000030  0067BC      33C6       0  CODE    
                text22                         0067BC  000036  0067F2      33DE       0  CODE    
                text20                         0067F2  000040  006832      33F9       0  CODE    
                text6                          006832  000042  006874      3419       0  CODE    
                text11                         006874  000046  0068BA      343A       0  CODE    
                text5                          0068BA  000052  00690C      345D       0  CODE    
                text21                         00690C  000084  006990      3486       0  CODE    
                text12                         006990  000096  006A26      34C8       0  CODE    
                text4                          006A26  0000A0  006AC6      3513       0  CODE    
                text1                          006AC6  000106  006BCC      3563       0  CODE    
                text0                          006BCC  000382  006F4E      35E6       0  CODE    
                mediumconst                    006F4E  0010B2  008000      37A7       0  MEDIUMCO
                idloc                          200000  000008  200008    200000       0  IDLOC   
                config                         300000  00000E  30000E    300000       0  CONFIG  


UNUSED ADDRESS RANGES

        Name                Unused          Largest block    Delta
        BANK0            000060-0000FF               A0
        BANK1            000100-0001FF              100
        BANK2            000200-0002FF              100
        BANK3            000300-0003FF              100
        BANK4            000400-0004FF              100
        BANK5            000500-0005FF              100
        BANK6            000600-0006FF              100
        BANK7            000700-0007FF              100
        BIGRAM           000030-0007FF              7D0
        CODE             001004-006653             5650
        COMRAM           000030-00005F               30
        CONST            001004-006653             5650
        EEDATA           F00000-F000FF              100
        FARRAM           000000-000000                1
        MEDIUMCONST      001004-006653             5650
        RAM              000060-0007FF              100
        SFR              000F60-000FFF               A0
        SMALLCONST       001004-006653              100
        STACK            000060-0007FF              7A0

                                  Symbol Table

?___awdiv                            cstackCOMRAM 000007
?___wmul                             cstackCOMRAM 000001
_LATBbits                            (abs)        000F8A
_PIR1bits                            (abs)        000F9E
_PIR2bits                            (abs)        000FA1
_SSPBUF                              (abs)        000FC9
_SSPCON1                             (abs)        000FC6
_SSPCON1bits                         (abs)        000FC6
_SSPCON2                             (abs)        000FC5
_SSPCON2bits                         (abs)        000FC5
_SSPSTAT                             (abs)        000FC7
_SSPSTATbits                         (abs)        000FC7
_TRISBbits                           (abs)        000F93
__CFG_BOR$ON                         (abs)        000000
__CFG_BORV$3                         (abs)        000000
__CFG_CP0$OFF                        (abs)        000000
__CFG_CP1$OFF                        (abs)        000000
__CFG_CPB$OFF                        (abs)        000000
__CFG_CPUDIV$OSC1_PLL2               (abs)        000000
__CFG_EBTR0$OFF                      (abs)        000000
__CFG_EBTR1$OFF                      (abs)        000000
__CFG_EBTRB$OFF                      (abs)        000000
__CFG_FCMEN$OFF                      (abs)        000000
__CFG_FOSC$HS                        (abs)        000000
__CFG_IESO$OFF                       (abs)        000000
__CFG_LPT1OSC$OFF                    (abs)        000000
__CFG_LVP$OFF                        (abs)        000000
__CFG_MCLRE$ON                       (abs)        000000
__CFG_PBADEN$OFF                     (abs)        000000
__CFG_PLLDIV$5                       (abs)        000000
__CFG_PWRT$OFF                       (abs)        000000
__CFG_STVREN$ON                      (abs)        000000
__CFG_USBDIV$2                       (abs)        000000
__CFG_VREGEN$ON                      (abs)        000000
__CFG_WDT$OFF                        (abs)        000000
__CFG_WDTPS$32768                    (abs)        000000
__CFG_WRT0$OFF                       (abs)        000000
__CFG_WRT1$OFF                       (abs)        000000
__CFG_WRTB$OFF                       (abs)        000000
__CFG_WRTC$OFF                       (abs)        000000
__CFG_XINST$OFF                      (abs)        000000
__HRAM                               (abs)        000000
__Habs1                              abs1         000000
__Hbank0                             bank0        000000
__Hbank1                             bank1        000000
__Hbank2                             bank2        000000
__Hbank3                             bank3        000000
__Hbank4                             bank4        000000
__Hbank5                             bank5        000000
__Hbank6                             bank6        000000
__Hbank7                             bank7        000000
__Hbigbss                            bigbss       000000
__Hbigdata                           bigdata      000000
__Hbigram                            bigram       000000
__Hbss                               bss          000000
__HbssCOMRAM                         bssCOMRAM    000000
__Hcinit                             cinit        000000
__Hclrtext                           clrtext      000000
__Hcomram                            comram       000000
__Hconfig                            config       30000E
__Hconst                             const        000000
__HcstackCOMRAM                      cstackCOMRAM 000000
__Hdata                              data         000000
__Heeprom_data                       eeprom_data  000000
__Hend_init                          end_init     001004
__Hfarbss                            farbss       000000
__Hfardata                           fardata      000000
__Hibigdata                          ibigdata     000000
__Hidata                             idata        000000
__Hidloc                             idloc        200008
__Hifardata                          ifardata     000000
__Hinit                              init         001000
__Hintcode                           intcode      001000
__Hintcode_body                      intcode_body 000000
__Hintcodelo                         intcodelo    001000
__Hintentry                          intentry     000000
__Hintret                            intret       000000
__Hintsave_regs                      intsave_regs 000000
__Hirdata                            irdata       000000
__Hmediumconst                       mediumconst  008000
__HnvFARRAM                          nvFARRAM     000000
__Hnvbit                             nvbit        000000
__Hnvrram                            nvrram       000000
__Hparam                             rparam       000000
__Hpowerup                           powerup      001000
__Hram                               ram          000000
__Hramtop                            ramtop       000800
__Hrbit                              rbit         000000
__Hrbss                              rbss         000000
__Hrdata                             rdata        000000
__Hreset_vec                         reset_vec    001000
__Hrparam                            rparam       000000
__Hsfr                               sfr          000000
__Hsmallconst                        smallconst   000000
__Hspace_0                           (abs)        30000E
__Hspace_1                           (abs)        000030
__Hspace_2                           (abs)        000000
__Hstack                             stack        000000
__Hstruct                            struct       000000
__Htemp                              temp         000000
__Htext                              text         000000
__Htext0                             text0        000000
__Htext1                             text1        000000
__Htext10                            text10       000000
__Htext11                            text11       000000
__Htext12                            text12       000000
__Htext13                            text13       000000
__Htext14                            text14       000000
__Htext15                            text15       000000
__Htext16                            text16       000000
__Htext17                            text17       000000
__Htext18                            text18       000000
__Htext19                            text19       000000
__Htext2                             text2        000000
__Htext20                            text20       000000
__Htext21                            text21       000000
__Htext22                            text22       000000
__Htext23                            text23       000000
__Htext3                             text3        000000
__Htext4                             text4        000000
__Htext5                             text5        000000
__Htext6                             text6        000000
__Htext7                             text7        000000
__Htext8                             text8        000000
__Htext9                             text9        000000
__LRAM                               (abs)        000001
__Labs1                              abs1         000000
__Lbank0                             bank0        000000
__Lbank1                             bank1        000000
__Lbank2                             bank2        000000
__Lbank3                             bank3        000000
__Lbank4                             bank4        000000
__Lbank5                             bank5        000000
__Lbank6                             bank6        000000
__Lbank7                             bank7        000000
__Lbigbss                            bigbss       000000
__Lbigdata                           bigdata      000000
__Lbigram                            bigram       000000
__Lbss                               bss          000000
__LbssCOMRAM                         bssCOMRAM    000000
__Lcinit                             cinit        000000
__Lclrtext                           clrtext      000000
__Lcomram                            comram       000000
__Lconfig                            config       300000
__Lconst                             const        000000
__LcstackCOMRAM                      cstackCOMRAM 000000
__Ldata                              data         000000
__Leeprom_data                       eeprom_data  000000
__Lend_init                          end_init     001000
__Lfarbss                            farbss       000000
__Lfardata                           fardata      000000
__Libigdata                          ibigdata     000000
__Lidata                             idata        000000
__Lidloc                             idloc        200000
__Lifardata                          ifardata     000000
__Linit                              init         001000
__Lintcode                           intcode      001000
__Lintcode_body                      intcode_body 000000
__Lintcodelo                         intcodelo    001000
__Lintentry                          intentry     000000
__Lintret                            intret       000000
__Lintsave_regs                      intsave_regs 000000
__Lirdata                            irdata       000000
__Lmediumconst                       mediumconst  006F4E
__LnvFARRAM                          nvFARRAM     000000
__Lnvbit                             nvbit        000000
__Lnvrram                            nvrram       000000
__Lparam                             rparam       000000
__Lpowerup                           powerup      001000
__Lram                               ram          000000
__Lramtop                            ramtop       000800
__Lrbit                              rbit         000000
__Lrbss                              rbss         000000
__Lrdata                             rdata        000000
__Lreset_vec                         reset_vec    001000
__Lrparam                            rparam       000000
__Lsfr                               sfr          000000
__Lsmallconst                        smallconst   000000
__Lspace_0                           (abs)        000000
__Lspace_1                           (abs)        000000
__Lspace_2                           (abs)        000000
__Lstack                             stack        000000
__Lstruct                            struct       000000
__Ltemp                              temp         000000
__Ltext                              text         000000
__Ltext0                             text0        000000
__Ltext1                             text1        000000
__Ltext10                            text10       000000
__Ltext11                            text11       000000
__Ltext12                            text12       000000
__Ltext13                            text13       000000
__Ltext14                            text14       000000
__Ltext15                            text15       000000
__Ltext16                            text16       000000
__Ltext17                            text17       000000
__Ltext18                            text18       000000
__Ltext19                            text19       000000
__Ltext2                             text2        000000
__Ltext20                            text20       000000
__Ltext21                            text21       000000
__Ltext22                            text22       000000
__Ltext23                            text23       000000
__Ltext3                             text3        000000
__Ltext4                             text4        000000
__Ltext5                             text5        000000
__Ltext6                             text6        000000
__Ltext7                             text7        000000
__Ltext8                             text8        000000
__Ltext9                             text9        000000
__S0                                 (abs)        30000E
__S1                                 (abs)        000030
__S2                                 (abs)        000000
___awdiv                             text21       00690C
___awdiv@counter                     cstackCOMRAM 00000B
___awdiv@dividend                    cstackCOMRAM 000007
___awdiv@divisor                     cstackCOMRAM 000009
___awdiv@quotient                    cstackCOMRAM 00000D
___awdiv@sign                        cstackCOMRAM 00000C
___inthi_sp                          stack        000000
___intlo_sp                          stack        000000
___param_bank                        (abs)        000010
___rparam_used                       (abs)        000001
___sp                                stack        000000
___wmul                              text23       0066EC
___wmul@multiplicand                 cstackCOMRAM 000003
___wmul@multiplier                   cstackCOMRAM 000001
___wmul@product                      cstackCOMRAM 000005
__accesstop                          (abs)        000060
__activetblptr                       (abs)        000002
__end_of___awdiv                     text21       006990
__end_of___wmul                      text23       006712
__end_of__initialization             cinit        0066E2
__end_of_delay_ms                    text22       0067F2
__end_of_img0_128x64c1               mediumconst  007B8D
__end_of_img1_128x64c1               mediumconst  007F8D
__end_of_main                        text0        006F4E
__end_of_ssd1306_char_font6x8        text6        006874
__end_of_ssd1306_draw_bmp            text12       006A26
__end_of_ssd1306_fill                text10       0066C0
__end_of_ssd1306_fill2               text9        0066D6
__end_of_ssd1306_fill4               text11       0068BA
__end_of_ssd1306_init                text7        00678C
__end_of_ssd1306_init_sequence       mediumconst  007783
__end_of_ssd1306_numdec_font6x8      text3        0067BC
__end_of_ssd1306_numdecp_font6x8     text2        006738
__end_of_ssd1306_send_byte           text20       006832
__end_of_ssd1306_send_command        text8        0066AA
__end_of_ssd1306_send_command_start  text15       006698
__end_of_ssd1306_send_command_stop   text14       006660
__end_of_ssd1306_send_data_start     text18       006686
__end_of_ssd1306_send_data_stop      text16       00665A
__end_of_ssd1306_setpos              text13       006760
__end_of_ssd1306_string_font6x8      text5        00690C
__end_of_ssd1306_string_font8x16xy   text1        006BCC
__end_of_ssd1306_xfer_start          text19       00666A
__end_of_ssd1306_xfer_stop           text17       006674
__end_of_ssd1306xled_font6x8         mediumconst  007767
__end_of_ssd1306xled_font8x16        mediumconst  00753F
__end_of_usint2decascii              text4        006AC6
__end_ofusint2decascii@F38           mediumconst  00778D
__initialization                     cinit        0066D6
__mediumconst                        mediumconst  006F4E
__pbssCOMRAM                         bssCOMRAM    00002A
__pcinit                             cinit        0066D6
__pcstackCOMRAM                      cstackCOMRAM 000001
__pmediumconst                       mediumconst  006F4E
__ptext0                             text0        006BCC
__ptext1                             text1        006AC6
__ptext10                            text10       0066AA
__ptext11                            text11       006874
__ptext12                            text12       006990
__ptext13                            text13       006738
__ptext14                            text14       00665A
__ptext15                            text15       006686
__ptext16                            text16       006654
__ptext17                            text17       00666A
__ptext18                            text18       006674
__ptext19                            text19       006660
__ptext2                             text2        006712
__ptext20                            text20       0067F2
__ptext21                            text21       00690C
__ptext22                            text22       0067BC
__ptext23                            text23       0066EC
__ptext3                             text3        00678C
__ptext4                             text4        006A26
__ptext5                             text5        0068BA
__ptext6                             text6        006832
__ptext7                             text7        006760
__ptext8                             text8        006698
__ptext9                             text9        0066C0
__ramtop                             ramtop       000800
__size_of___awdiv                    (abs)        000000
__size_of___wmul                     (abs)        000000
__size_of_delay_ms                   (abs)        000000
__size_of_main                       (abs)        000000
__size_of_ssd1306_char_font6x8       (abs)        000000
__size_of_ssd1306_draw_bmp           (abs)        000000
__size_of_ssd1306_fill               (abs)        000000
__size_of_ssd1306_fill2              (abs)        000000
__size_of_ssd1306_fill4              (abs)        000000
__size_of_ssd1306_init               (abs)        000000
__size_of_ssd1306_numdec_font6x8     (abs)        000000
__size_of_ssd1306_numdecp_font6x8    (abs)        000000
__size_of_ssd1306_send_byte          (abs)        000000
__size_of_ssd1306_send_command       (abs)        000000
__size_of_ssd1306_send_command_start (abs)        000000
__size_of_ssd1306_send_command_stop  (abs)        000000
__size_of_ssd1306_send_data_start    (abs)        000000
__size_of_ssd1306_send_data_stop     (abs)        000000
__size_of_ssd1306_setpos             (abs)        000000
__size_of_ssd1306_string_font6x8     (abs)        000000
__size_of_ssd1306_string_font8x16xy  (abs)        000000
__size_of_ssd1306_xfer_start         (abs)        000000
__size_of_ssd1306_xfer_stop          (abs)        000000
__size_of_usint2decascii             (abs)        000000
__smallconst                         smallconst   000000
_delay_ms                            text22       0067BC
_img0_128x64c1                       mediumconst  00778D
_img1_128x64c1                       mediumconst  007B8D
_main                                text0        006BCC
_ssd1306_char_font6x8                text6        006832
_ssd1306_draw_bmp                    text12       006990
_ssd1306_fill                        text10       0066AA
_ssd1306_fill2                       text9        0066C0
_ssd1306_fill4                       text11       006874
_ssd1306_init                        text7        006760
_ssd1306_init_sequence               mediumconst  007767
_ssd1306_numdec_buffer               bssCOMRAM    00002A
_ssd1306_numdec_font6x8              text3        00678C
_ssd1306_numdecp_font6x8             text2        006712
_ssd1306_send_byte                   text20       0067F2
_ssd1306_send_command                text8        006698
_ssd1306_send_command_start          text15       006686
_ssd1306_send_command_stop           text14       00665A
_ssd1306_send_data_start             text18       006674
_ssd1306_send_data_stop              text16       006654
_ssd1306_setpos                      text13       006738
_ssd1306_string_font6x8              text5        0068BA
_ssd1306_string_font8x16xy           text1        006AC6
_ssd1306_xfer_start                  text19       006660
_ssd1306_xfer_stop                   text17       00666A
_ssd1306xled_font6x8                 mediumconst  00753F
_ssd1306xled_font8x16                mediumconst  006F4F
_usint2decascii                      text4        006A26
delay_ms@n                           cstackCOMRAM 000001
end_of_initialization                cinit        0066E2
intlevel0                            text         000000
intlevel1                            text         000000
intlevel2                            text         000000
intlevel3                            text         000000
main@i                               cstackCOMRAM 000022
main@i_1250                          cstackCOMRAM 000023
main@i_1254                          cstackCOMRAM 000024
main@i_1257                          cstackCOMRAM 000025
main@j                               cstackCOMRAM 000028
main@j_1253                          cstackCOMRAM 000029
main@n1                              cstackCOMRAM 00001D
main@n2                              cstackCOMRAM 00001F
main@n3                              cstackCOMRAM 000026
main@p                               cstackCOMRAM 000021
ssd1306_char_font6x8@c               cstackCOMRAM 000007
ssd1306_char_font6x8@ch              cstackCOMRAM 000006
ssd1306_char_font6x8@i               cstackCOMRAM 000008
ssd1306_draw_bmp@bitmap              cstackCOMRAM 000012
ssd1306_draw_bmp@j                   cstackCOMRAM 000016
ssd1306_draw_bmp@x                   cstackCOMRAM 000018
ssd1306_draw_bmp@x0                  cstackCOMRAM 000019
ssd1306_draw_bmp@x1                  cstackCOMRAM 000010
ssd1306_draw_bmp@y                   cstackCOMRAM 00001A
ssd1306_draw_bmp@y0                  cstackCOMRAM 00000F
ssd1306_draw_bmp@y1                  cstackCOMRAM 000011
ssd1306_fill2@p1                     cstackCOMRAM 00000F
ssd1306_fill2@p2                     cstackCOMRAM 00000E
ssd1306_fill4@i                      cstackCOMRAM 00000C
ssd1306_fill4@p1                     cstackCOMRAM 00000B
ssd1306_fill4@p2                     cstackCOMRAM 000008
ssd1306_fill4@p3                     cstackCOMRAM 000009
ssd1306_fill4@p4                     cstackCOMRAM 00000A
ssd1306_fill@p                       cstackCOMRAM 00000E
ssd1306_init@i                       cstackCOMRAM 000007
ssd1306_numdec_font6x8@digits        cstackCOMRAM 000016
ssd1306_numdec_font6x8@num           cstackCOMRAM 000014
ssd1306_numdecp_font6x8@num          cstackCOMRAM 000014
ssd1306_send_byte@byte               cstackCOMRAM 000004
ssd1306_send_byte@i                  cstackCOMRAM 000005
ssd1306_send_command@command         cstackCOMRAM 000006
ssd1306_setpos@x                     cstackCOMRAM 000007
ssd1306_setpos@y                     cstackCOMRAM 000006
ssd1306_string_font6x8@s             cstackCOMRAM 000009
ssd1306_string_font8x16xy@ch         cstackCOMRAM 00000D
ssd1306_string_font8x16xy@i          cstackCOMRAM 000010
ssd1306_string_font8x16xy@i_1458     cstackCOMRAM 000011
ssd1306_string_font8x16xy@j          cstackCOMRAM 00000E
ssd1306_string_font8x16xy@s          cstackCOMRAM 000009
ssd1306_string_font8x16xy@x          cstackCOMRAM 00000F
ssd1306_string_font8x16xy@y          cstackCOMRAM 000008
stackhi                              (abs)        0007FF
stacklo                              (abs)        000060
start                                init         001000
start_initialization                 cinit        0066D6
usint2decascii@F38                   mediumconst  007783
usint2decascii@buffer                cstackCOMRAM 000003
usint2decascii@digit                 cstackCOMRAM 000012
usint2decascii@digits                cstackCOMRAM 000011
usint2decascii@num                   cstackCOMRAM 000001
usint2decascii@pos                   cstackCOMRAM 000013
usint2decascii@powers                cstackCOMRAM 000007


FUNCTION INFORMATION:

 *************** function _main *****************
 Defined at:
		line 18 in file "main_OLED.c"
 Parameters:    Size  Location     Type
		None
 Auto vars:     Size  Location     Type
  i               1   35[COMRAM] unsigned char 
  i               1   34[COMRAM] unsigned char 
  i               1   36[COMRAM] unsigned char 
  j               1   40[COMRAM] unsigned char 
  j               1   39[COMRAM] unsigned char 
  i               1   33[COMRAM] unsigned char 
  n3              2   37[COMRAM] int 
  n2              2   30[COMRAM] int 
  n1              2   28[COMRAM] int 
  p               1   32[COMRAM] unsigned char 
 Return value:  Size  Location     Type
		None               void
 Registers used:
		wreg, fsr0l, fsr0h, fsr2l, fsr2h, status,2, status,0, tblptrl, tblptrh, tblptru, prodl, prodh, cstack
 Tracked objects:
		On entry : 
		On exit  : 
		Unchanged: 
 Data sizes:     COMRAM   BANK0   BANK1   BANK2   BANK3   BANK4   BANK5   BANK6   BANK7
      Params:         0       0       0       0       0       0       0       0       0
      Locals:        13       0       0       0       0       0       0       0       0
      Temps:          2       0       0       0       0       0       0       0       0
      Totals:        15       0       0       0       0       0       0       0       0
Total ram usage:       15 bytes
 Hardware stack levels required when called:    5
 This function calls:
		___awdiv
		___wmul
		_delay_ms
		_ssd1306_draw_bmp
		_ssd1306_fill
		_ssd1306_fill2
		_ssd1306_fill4
		_ssd1306_init
		_ssd1306_numdec_font6x8
		_ssd1306_numdecp_font6x8
		_ssd1306_setpos
		_ssd1306_string_font6x8
		_ssd1306_string_font8x16xy
 This function is called by:
		Startup code after reset
 This function uses a non-reentrant model


 *************** function _ssd1306_string_font8x16xy *****************
 Defined at:
		line 49 in file "ssd1306xled8x16.c"
 Parameters:    Size  Location     Type
  x               1    wreg     unsigned char 
  y               1    7[COMRAM] unsigned char 
  s               2    8[COMRAM] PTR unsigned char 
		 -> STR_6(9), 
 Auto vars:     Size  Location     Type
  x               1   14[COMRAM] unsigned char 
  i               1   16[COMRAM] unsigned char 
  i               1   15[COMRAM] unsigned char 
  j               1   13[COMRAM] unsigned char 
  ch              1   12[COMRAM] unsigned char 
 Return value:  Size  Location     Type
		None               void
 Registers used:
		wreg, status,2, status,0, tblptrl, tblptrh, tblptru, prodl, prodh, cstack
 Tracked objects:
		On entry : 
		On exit  : 
		Unchanged: 
 Data sizes:     COMRAM   BANK0   BANK1   BANK2   BANK3   BANK4   BANK5   BANK6   BANK7
      Params:         3       0       0       0       0       0       0       0       0
      Locals:         5       0       0       0       0       0       0       0       0
      Temps:          2       0       0       0       0       0       0       0       0
      Totals:        10       0       0       0       0       0       0       0       0
Total ram usage:       10 bytes
 Hardware stack levels used:    1
 Hardware stack levels required when called:    3
 This function calls:
		_ssd1306_send_byte
		_ssd1306_send_data_start
		_ssd1306_send_data_stop
		_ssd1306_setpos
 This function is called by:
		_main
 This function uses a non-reentrant model


 *************** function _ssd1306_numdecp_font6x8 *****************
 Defined at:
		line 229 in file "ssd1306xled.c"
 Parameters:    Size  Location     Type
  num             2   19[COMRAM] int 
 Auto vars:     Size  Location     Type
		None
 Return value:  Size  Location     Type
		None               void
 Registers used:
		wreg, fsr0l, fsr0h, fsr2l, fsr2h, status,2, status,0, tblptrl, tblptrh, tblptru, prodl, prodh, cstack
 Tracked objects:
		On entry : 
		On exit  : 
		Unchanged: 
 Data sizes:     COMRAM   BANK0   BANK1   BANK2   BANK3   BANK4   BANK5   BANK6   BANK7
      Params:         2       0       0       0       0       0       0       0       0
      Locals:         0       0       0       0       0       0       0       0       0
      Temps:          0       0       0       0       0       0       0       0       0
      Totals:         2       0       0       0       0       0       0       0       0
Total ram usage:        2 bytes
 Hardware stack levels used:    1
 Hardware stack levels required when called:    4
 This function calls:
		_ssd1306_string_font6x8
		_usint2decascii
 This function is called by:
		_main
 This function uses a non-reentrant model


 *************** function _ssd1306_numdec_font6x8 *****************
 Defined at:
		line 223 in file "ssd1306xled.c"
 Parameters:    Size  Location     Type
  num             2   19[COMRAM] int 
 Auto vars:     Size  Location     Type
  digits          1   21[COMRAM] unsigned char 
 Return value:  Size  Location     Type
		None               void
 Registers used:
		wreg, fsr0l, fsr0h, fsr2l, fsr2h, status,2, status,0, tblptrl, tblptrh, tblptru, prodl, prodh, cstack
 Tracked objects:
		On entry : 
		On exit  : 
		Unchanged: 
 Data sizes:     COMRAM   BANK0   BANK1   BANK2   BANK3   BANK4   BANK5   BANK6   BANK7
      Params:         2       0       0       0       0       0       0       0       0
      Locals:         1       0       0       0       0       0       0       0       0
      Temps:          0       0       0       0       0       0       0       0       0
      Totals:         3       0       0       0       0       0       0       0       0
Total ram usage:        3 bytes
 Hardware stack levels used:    1
 Hardware stack levels required when called:    4
 This function calls:
		_ssd1306_string_font6x8
		_usint2decascii
 This function is called by:
		_main
 This function uses a non-reentrant model


 *************** function _usint2decascii *****************
 Defined at:
		line 27 in file "num2str.c"
 Parameters:    Size  Location     Type
  num             2    0[COMRAM] int 
  buffer          2    2[COMRAM] PTR unsigned char 
		 -> ssd1306_numdec_buffer(6), 
 Auto vars:     Size  Location     Type
  pos             1   18[COMRAM] unsigned char 
  powers         10    6[COMRAM] const unsigned short [5]
  digit           1   17[COMRAM] unsigned char 
  digits          1   16[COMRAM] unsigned char 
 Return value:  Size  Location     Type
                  1    wreg      unsigned char 
 Registers used:
		wreg, fsr2l, fsr2h, status,2, status,0, tblptrl, tblptrh, tblptru, prodl, prodh
 Tracked objects:
		On entry : 
		On exit  : 
		Unchanged: 
 Data sizes:     COMRAM   BANK0   BANK1   BANK2   BANK3   BANK4   BANK5   BANK6   BANK7
      Params:         4       0       0       0       0       0       0       0       0
      Locals:        13       0       0       0       0       0       0       0       0
      Temps:          2       0       0       0       0       0       0       0       0
      Totals:        19       0       0       0       0       0       0       0       0
Total ram usage:       19 bytes
 Hardware stack levels used:    1
 This function calls:
		Nothing
 This function is called by:
		_ssd1306_numdec_font6x8
		_ssd1306_numdecp_font6x8
 This function uses a non-reentrant model


 *************** function _ssd1306_string_font6x8 *****************
 Defined at:
		line 215 in file "ssd1306xled.c"
 Parameters:    Size  Location     Type
  s               2    8[COMRAM] PTR unsigned char 
		 -> ssd1306_numdec_buffer(6), STR_9(20), STR_8(64), STR_7(8), 
		 -> STR_5(12), STR_4(3), STR_3(3), STR_2(2), 
		 -> STR_1(2), 
 Auto vars:     Size  Location     Type
		None
 Return value:  Size  Location     Type
		None               void
 Registers used:
		wreg, fsr0l, fsr0h, status,2, status,0, tblptrl, tblptrh, tblptru, prodl, prodh, cstack
 Tracked objects:
		On entry : 
		On exit  : 
		Unchanged: 
 Data sizes:     COMRAM   BANK0   BANK1   BANK2   BANK3   BANK4   BANK5   BANK6   BANK7
      Params:         2       0       0       0       0       0       0       0       0
      Locals:         0       0       0       0       0       0       0       0       0
      Temps:          0       0       0       0       0       0       0       0       0
      Totals:         2       0       0       0       0       0       0       0       0
Total ram usage:        2 bytes
 Hardware stack levels used:    1
 Hardware stack levels required when called:    3
 This function calls:
		_ssd1306_char_font6x8
 This function is called by:
		_main
		_ssd1306_numdec_font6x8
		_ssd1306_numdecp_font6x8
 This function uses a non-reentrant model


 *************** function _ssd1306_char_font6x8 *****************
 Defined at:
		line 205 in file "ssd1306xled.c"
 Parameters:    Size  Location     Type
  ch              1    wreg     unsigned char 
 Auto vars:     Size  Location     Type
  ch              1    5[COMRAM] unsigned char 
  i               1    7[COMRAM] unsigned char 
  c               1    6[COMRAM] unsigned char 
 Return value:  Size  Location     Type
		None               void
 Registers used:
		wreg, status,2, status,0, tblptrl, tblptrh, tblptru, prodl, prodh, cstack
 Tracked objects:
		On entry : 
		On exit  : 
		Unchanged: 
 Data sizes:     COMRAM   BANK0   BANK1   BANK2   BANK3   BANK4   BANK5   BANK6   BANK7
      Params:         0       0       0       0       0       0       0       0       0
      Locals:         3       0       0       0       0       0       0       0       0
      Temps:          0       0       0       0       0       0       0       0       0
      Totals:         3       0       0       0       0       0       0       0       0
Total ram usage:        3 bytes
 Hardware stack levels used:    1
 Hardware stack levels required when called:    2
 This function calls:
		_ssd1306_send_byte
		_ssd1306_send_data_start
		_ssd1306_send_data_stop
 This function is called by:
		_ssd1306_string_font6x8
 This function uses a non-reentrant model


 *************** function _ssd1306_init *****************
 Defined at:
		line 162 in file "ssd1306xled.c"
 Parameters:    Size  Location     Type
		None
 Auto vars:     Size  Location     Type
  i               1    6[COMRAM] unsigned char 
 Return value:  Size  Location     Type
		None               void
 Registers used:
		wreg, status,2, status,0, tblptrl, tblptrh, tblptru, prodl, prodh, cstack
 Tracked objects:
		On entry : 
		On exit  : 
		Unchanged: 
 Data sizes:     COMRAM   BANK0   BANK1   BANK2   BANK3   BANK4   BANK5   BANK6   BANK7
      Params:         0       0       0       0       0       0       0       0       0
      Locals:         1       0       0       0       0       0       0       0       0
      Temps:          0       0       0       0       0       0       0       0       0
      Totals:         1       0       0       0       0       0       0       0       0
Total ram usage:        1 bytes
 Hardware stack levels used:    1
 Hardware stack levels required when called:    3
 This function calls:
		_ssd1306_send_command
 This function is called by:
		_main
 This function uses a non-reentrant model


 *************** function _ssd1306_send_command *****************
 Defined at:
		line 132 in file "ssd1306xled.c"
 Parameters:    Size  Location     Type
  command         1    wreg     unsigned char 
 Auto vars:     Size  Location     Type
  command         1    5[COMRAM] unsigned char 
 Return value:  Size  Location     Type
		None               void
 Registers used:
		wreg, status,2, status,0, cstack
 Tracked objects:
		On entry : 
		On exit  : 
		Unchanged: 
 Data sizes:     COMRAM   BANK0   BANK1   BANK2   BANK3   BANK4   BANK5   BANK6   BANK7
      Params:         0       0       0       0       0       0       0       0       0
      Locals:         1       0       0       0       0       0       0       0       0
      Temps:          0       0       0       0       0       0       0       0       0
      Totals:         1       0       0       0       0       0       0       0       0
Total ram usage:        1 bytes
 Hardware stack levels used:    1
 Hardware stack levels required when called:    2
 This function calls:
		_ssd1306_send_byte
		_ssd1306_send_command_start
		_ssd1306_send_command_stop
 This function is called by:
		_ssd1306_init
 This function uses a non-reentrant model


 *************** function _ssd1306_fill2 *****************
 Defined at:
		line 195 in file "ssd1306xled.c"
 Parameters:    Size  Location     Type
  p1              1    wreg     unsigned char 
  p2              1   13[COMRAM] unsigned char 
 Auto vars:     Size  Location     Type
  p1              1   14[COMRAM] unsigned char 
 Return value:  Size  Location     Type
		None               void
 Registers used:
		wreg, status,2, status,0, cstack
 Tracked objects:
		On entry : 
		On exit  : 
		Unchanged: 
 Data sizes:     COMRAM   BANK0   BANK1   BANK2   BANK3   BANK4   BANK5   BANK6   BANK7
      Params:         1       0       0       0       0       0       0       0       0
      Locals:         1       0       0       0       0       0       0       0       0
      Temps:          0       0       0       0       0       0       0       0       0
      Totals:         2       0       0       0       0       0       0       0       0
Total ram usage:        2 bytes
 Hardware stack levels used:    1
 Hardware stack levels required when called:    4
 This function calls:
		_ssd1306_fill4
 This function is called by:
		_main
 This function uses a non-reentrant model


 *************** function _ssd1306_fill *****************
 Defined at:
		line 199 in file "ssd1306xled.c"
 Parameters:    Size  Location     Type
  p               1    wreg     unsigned char 
 Auto vars:     Size  Location     Type
  p               1   13[COMRAM] unsigned char 
 Return value:  Size  Location     Type
		None               void
 Registers used:
		wreg, status,2, status,0, cstack
 Tracked objects:
		On entry : 
		On exit  : 
		Unchanged: 
 Data sizes:     COMRAM   BANK0   BANK1   BANK2   BANK3   BANK4   BANK5   BANK6   BANK7
      Params:         0       0       0       0       0       0       0       0       0
      Locals:         1       0       0       0       0       0       0       0       0
      Temps:          0       0       0       0       0       0       0       0       0
      Totals:         1       0       0       0       0       0       0       0       0
Total ram usage:        1 bytes
 Hardware stack levels used:    1
 Hardware stack levels required when called:    4
 This function calls:
		_ssd1306_fill4
 This function is called by:
		_main
 This function uses a non-reentrant model


 *************** function _ssd1306_fill4 *****************
 Defined at:
		line 183 in file "ssd1306xled.c"
 Parameters:    Size  Location     Type
  p1              1    wreg     unsigned char 
  p2              1    7[COMRAM] unsigned char 
  p3              1    8[COMRAM] unsigned char 
  p4              1    9[COMRAM] unsigned char 
 Auto vars:     Size  Location     Type
  p1              1   10[COMRAM] unsigned char 
  i               2   11[COMRAM] int 
 Return value:  Size  Location     Type
		None               void
 Registers used:
		wreg, status,2, status,0, cstack
 Tracked objects:
		On entry : 
		On exit  : 
		Unchanged: 
 Data sizes:     COMRAM   BANK0   BANK1   BANK2   BANK3   BANK4   BANK5   BANK6   BANK7
      Params:         3       0       0       0       0       0       0       0       0
      Locals:         3       0       0       0       0       0       0       0       0
      Temps:          0       0       0       0       0       0       0       0       0
      Totals:         6       0       0       0       0       0       0       0       0
Total ram usage:        6 bytes
 Hardware stack levels used:    1
 Hardware stack levels required when called:    3
 This function calls:
		_ssd1306_send_byte
		_ssd1306_send_data_start
		_ssd1306_send_data_stop
		_ssd1306_setpos
 This function is called by:
		_main
		_ssd1306_fill2
		_ssd1306_fill
 This function uses a non-reentrant model


 *************** function _ssd1306_draw_bmp *****************
 Defined at:
		line 237 in file "ssd1306xled.c"
 Parameters:    Size  Location     Type
  x0              1    wreg     unsigned char 
  y0              1   14[COMRAM] unsigned char 
  x1              1   15[COMRAM] unsigned char 
  y1              1   16[COMRAM] unsigned char 
  bitmap          2   17[COMRAM] PTR const unsigned char 
		 -> img0_128x64c1(1024), img1_128x64c1(1024), 
 Auto vars:     Size  Location     Type
  x0              1   24[COMRAM] unsigned char 
  x               1   23[COMRAM] unsigned char 
  j               2   21[COMRAM] int 
  y               1   25[COMRAM] unsigned char 
 Return value:  Size  Location     Type
		None               void
 Registers used:
		wreg, status,2, status,0, tblptrl, tblptrh, tblptru, cstack
 Tracked objects:
		On entry : 
		On exit  : 
		Unchanged: 
 Data sizes:     COMRAM   BANK0   BANK1   BANK2   BANK3   BANK4   BANK5   BANK6   BANK7
      Params:         5       0       0       0       0       0       0       0       0
      Locals:         5       0       0       0       0       0       0       0       0
      Temps:          2       0       0       0       0       0       0       0       0
      Totals:        12       0       0       0       0       0       0       0       0
Total ram usage:       12 bytes
 Hardware stack levels used:    1
 Hardware stack levels required when called:    3
 This function calls:
		___awdiv
		_ssd1306_send_byte
		_ssd1306_send_data_start
		_ssd1306_send_data_stop
		_ssd1306_setpos
 This function is called by:
		_main
 This function uses a non-reentrant model


 *************** function _ssd1306_setpos *****************
 Defined at:
		line 174 in file "ssd1306xled.c"
 Parameters:    Size  Location     Type
  x               1    wreg     unsigned char 
  y               1    5[COMRAM] unsigned char 
 Auto vars:     Size  Location     Type
  x               1    6[COMRAM] unsigned char 
 Return value:  Size  Location     Type
		None               void
 Registers used:
		wreg, status,2, status,0, cstack
 Tracked objects:
		On entry : 
		On exit  : 
		Unchanged: 
 Data sizes:     COMRAM   BANK0   BANK1   BANK2   BANK3   BANK4   BANK5   BANK6   BANK7
      Params:         1       0       0       0       0       0       0       0       0
      Locals:         1       0       0       0       0       0       0       0       0
      Temps:          0       0       0       0       0       0       0       0       0
      Totals:         2       0       0       0       0       0       0       0       0
Total ram usage:        2 bytes
 Hardware stack levels used:    1
 Hardware stack levels required when called:    2
 This function calls:
		_ssd1306_send_byte
		_ssd1306_send_command_start
		_ssd1306_send_command_stop
 This function is called by:
		_main
		_ssd1306_fill4
		_ssd1306_draw_bmp
		_ssd1306_string_font8x16xy
 This function uses a non-reentrant model


 *************** function _ssd1306_send_command_stop *****************
 Defined at:
		line 128 in file "ssd1306xled.c"
 Parameters:    Size  Location     Type
		None
 Auto vars:     Size  Location     Type
		None
 Return value:  Size  Location     Type
		None               void
 Registers used:
		cstack
 Tracked objects:
		On entry : 
		On exit  : 
		Unchanged: 
 Data sizes:     COMRAM   BANK0   BANK1   BANK2   BANK3   BANK4   BANK5   BANK6   BANK7
      Params:         0       0       0       0       0       0       0       0       0
      Locals:         0       0       0       0       0       0       0       0       0
      Temps:          0       0       0       0       0       0       0       0       0
      Totals:         0       0       0       0       0       0       0       0       0
Total ram usage:        0 bytes
 Hardware stack levels used:    1
 Hardware stack levels required when called:    1
 This function calls:
		_ssd1306_xfer_stop
 This function is called by:
		_ssd1306_send_command
		_ssd1306_setpos
 This function uses a non-reentrant model


 *************** function _ssd1306_send_command_start *****************
 Defined at:
		line 122 in file "ssd1306xled.c"
 Parameters:    Size  Location     Type
		None
 Auto vars:     Size  Location     Type
		None
 Return value:  Size  Location     Type
		None               void
 Registers used:
		wreg, status,2, status,0, cstack
 Tracked objects:
		On entry : 
		On exit  : 
		Unchanged: 
 Data sizes:     COMRAM   BANK0   BANK1   BANK2   BANK3   BANK4   BANK5   BANK6   BANK7
      Params:         0       0       0       0       0       0       0       0       0
      Locals:         0       0       0       0       0       0       0       0       0
      Temps:          0       0       0       0       0       0       0       0       0
      Totals:         0       0       0       0       0       0       0       0       0
Total ram usage:        0 bytes
 Hardware stack levels used:    1
 Hardware stack levels required when called:    1
 This function calls:
		_ssd1306_send_byte
		_ssd1306_xfer_start
 This function is called by:
		_ssd1306_send_command
		_ssd1306_setpos
 This function uses a non-reentrant model


 *************** function _ssd1306_send_data_stop *****************
 Defined at:
		line 146 in file "ssd1306xled.c"
 Parameters:    Size  Location     Type
		None
 Auto vars:     Size  Location     Type
		None
 Return value:  Size  Location     Type
		None               void
 Registers used:
		cstack
 Tracked objects:
		On entry : 
		On exit  : 
		Unchanged: 
 Data sizes:     COMRAM   BANK0   BANK1   BANK2   BANK3   BANK4   BANK5   BANK6   BANK7
      Params:         0       0       0       0       0       0       0       0       0
      Locals:         0       0       0       0       0       0       0       0       0
      Temps:          0       0       0       0       0       0       0       0       0
      Totals:         0       0       0       0       0       0       0       0       0
Total ram usage:        0 bytes
 Hardware stack levels used:    1
 Hardware stack levels required when called:    1
 This function calls:
		_ssd1306_xfer_stop
 This function is called by:
		_ssd1306_fill4
		_ssd1306_char_font6x8
		_ssd1306_draw_bmp
		_ssd1306_string_font8x16xy
 This function uses a non-reentrant model


 *************** function _ssd1306_xfer_stop *****************
 Defined at:
		line 86 in file "ssd1306xled.c"
 Parameters:    Size  Location     Type
		None
 Auto vars:     Size  Location     Type
		None
 Return value:  Size  Location     Type
		None               void
 Registers used:
		None
 Tracked objects:
		On entry : 
		On exit  : 
		Unchanged: 
 Data sizes:     COMRAM   BANK0   BANK1   BANK2   BANK3   BANK4   BANK5   BANK6   BANK7
      Params:         0       0       0       0       0       0       0       0       0
      Locals:         0       0       0       0       0       0       0       0       0
      Temps:          0       0       0       0       0       0       0       0       0
      Totals:         0       0       0       0       0       0       0       0       0
Total ram usage:        0 bytes
 Hardware stack levels used:    1
 This function calls:
		Nothing
 This function is called by:
		_ssd1306_send_command_stop
		_ssd1306_send_data_stop
 This function uses a non-reentrant model


 *************** function _ssd1306_send_data_start *****************
 Defined at:
		line 139 in file "ssd1306xled.c"
 Parameters:    Size  Location     Type
		None
 Auto vars:     Size  Location     Type
		None
 Return value:  Size  Location     Type
		None               void
 Registers used:
		wreg, status,2, status,0, cstack
 Tracked objects:
		On entry : 
		On exit  : 
		Unchanged: 
 Data sizes:     COMRAM   BANK0   BANK1   BANK2   BANK3   BANK4   BANK5   BANK6   BANK7
      Params:         0       0       0       0       0       0       0       0       0
      Locals:         0       0       0       0       0       0       0       0       0
      Temps:          0       0       0       0       0       0       0       0       0
      Totals:         0       0       0       0       0       0       0       0       0
Total ram usage:        0 bytes
 Hardware stack levels used:    1
 Hardware stack levels required when called:    1
 This function calls:
		_ssd1306_send_byte
		_ssd1306_xfer_start
 This function is called by:
		_ssd1306_fill4
		_ssd1306_char_font6x8
		_ssd1306_draw_bmp
		_ssd1306_string_font8x16xy
 This function uses a non-reentrant model


 *************** function _ssd1306_xfer_start *****************
 Defined at:
		line 74 in file "ssd1306xled.c"
 Parameters:    Size  Location     Type
		None
 Auto vars:     Size  Location     Type
		None
 Return value:  Size  Location     Type
		None               void
 Registers used:
		None
 Tracked objects:
		On entry : 
		On exit  : 
		Unchanged: 
 Data sizes:     COMRAM   BANK0   BANK1   BANK2   BANK3   BANK4   BANK5   BANK6   BANK7
      Params:         0       0       0       0       0       0       0       0       0
      Locals:         0       0       0       0       0       0       0       0       0
      Temps:          0       0       0       0       0       0       0       0       0
      Totals:         0       0       0       0       0       0       0       0       0
Total ram usage:        0 bytes
 Hardware stack levels used:    1
 This function calls:
		Nothing
 This function is called by:
		_ssd1306_send_command_start
		_ssd1306_send_data_start
 This function uses a non-reentrant model


 *************** function _ssd1306_send_byte *****************
 Defined at:
		line 98 in file "ssd1306xled.c"
 Parameters:    Size  Location     Type
  byte            1    wreg     unsigned char 
 Auto vars:     Size  Location     Type
  byte            1    3[COMRAM] unsigned char 
  i               1    4[COMRAM] unsigned char 
 Return value:  Size  Location     Type
		None               void
 Registers used:
		wreg, status,2, status,0
 Tracked objects:
		On entry : 
		On exit  : 
		Unchanged: 
 Data sizes:     COMRAM   BANK0   BANK1   BANK2   BANK3   BANK4   BANK5   BANK6   BANK7
      Params:         0       0       0       0       0       0       0       0       0
      Locals:         2       0       0       0       0       0       0       0       0
      Temps:          3       0       0       0       0       0       0       0       0
      Totals:         5       0       0       0       0       0       0       0       0
Total ram usage:        5 bytes
 Hardware stack levels used:    1
 This function calls:
		Nothing
 This function is called by:
		_ssd1306_send_command_start
		_ssd1306_send_command
		_ssd1306_send_data_start
		_ssd1306_setpos
		_ssd1306_fill4
		_ssd1306_char_font6x8
		_ssd1306_draw_bmp
		_ssd1306_string_font8x16xy
 This function uses a non-reentrant model


 *************** function ___awdiv *****************
 Defined at:
		line 8 in file "C:\Program Files\Microchip\xc8\v1.35\sources\common\awdiv.c"
 Parameters:    Size  Location     Type
  dividend        2    6[COMRAM] int 
  divisor         2    8[COMRAM] int 
 Auto vars:     Size  Location     Type
  quotient        2   12[COMRAM] int 
  sign            1   11[COMRAM] unsigned char 
  counter         1   10[COMRAM] unsigned char 
 Return value:  Size  Location     Type
                  2    6[COMRAM] int 
 Registers used:
		wreg, status,2, status,0
 Tracked objects:
		On entry : 
		On exit  : 
		Unchanged: 
 Data sizes:     COMRAM   BANK0   BANK1   BANK2   BANK3   BANK4   BANK5   BANK6   BANK7
      Params:         4       0       0       0       0       0       0       0       0
      Locals:         4       0       0       0       0       0       0       0       0
      Temps:          0       0       0       0       0       0       0       0       0
      Totals:         8       0       0       0       0       0       0       0       0
Total ram usage:        8 bytes
 Hardware stack levels used:    1
 This function calls:
		Nothing
 This function is called by:
		_main
		_ssd1306_draw_bmp
 This function uses a non-reentrant model


 *************** function _delay_ms *****************
 Defined at:
		line 146 in file "Alteri.h"
 Parameters:    Size  Location     Type
  n               4    0[COMRAM] long 
 Auto vars:     Size  Location     Type
		None
 Return value:  Size  Location     Type
		None               void
 Registers used:
		wreg, status,2, status,0
 Tracked objects:
		On entry : 
		On exit  : 
		Unchanged: 
 Data sizes:     COMRAM   BANK0   BANK1   BANK2   BANK3   BANK4   BANK5   BANK6   BANK7
      Params:         4       0       0       0       0       0       0       0       0
      Locals:         0       0       0       0       0       0       0       0       0
      Temps:          1       0       0       0       0       0       0       0       0
      Totals:         5       0       0       0       0       0       0       0       0
Total ram usage:        5 bytes
 Hardware stack levels used:    1
 This function calls:
		Nothing
 This function is called by:
		_main
 This function uses a non-reentrant model


 *************** function ___wmul *****************
 Defined at:
		line 15 in file "C:\Program Files\Microchip\xc8\v1.35\sources\common\Umul16.c"
 Parameters:    Size  Location     Type
  multiplier      2    0[COMRAM] unsigned int 
  multiplicand    2    2[COMRAM] unsigned int 
 Auto vars:     Size  Location     Type
  product         2    4[COMRAM] unsigned int 
 Return value:  Size  Location     Type
                  2    0[COMRAM] unsigned int 
 Registers used:
		wreg, status,2, status,0, prodl, prodh
 Tracked objects:
		On entry : 
		On exit  : 
		Unchanged: 
 Data sizes:     COMRAM   BANK0   BANK1   BANK2   BANK3   BANK4   BANK5   BANK6   BANK7
      Params:         4       0       0       0       0       0       0       0       0
      Locals:         2       0       0       0       0       0       0       0       0
      Temps:          0       0       0       0       0       0       0       0       0
      Totals:         6       0       0       0       0       0       0       0       0
Total ram usage:        6 bytes
 Hardware stack levels used:    1
 This function calls:
		Nothing
 This function is called by:
		_main
 This function uses a non-reentrant model



MODULE INFORMATION

Module		Function		Class		Link	Load	Size
num2str.c
		_usint2decascii		CODE           	6A26	0000	161

num2str.c estimated size: 161

ssd1306xled8x16.c
		_ssd1306_string_font8x16xy		CODE           	6AC6	0000	263

ssd1306xled8x16.c estimated size: 263

main_OLED.c
		_main          		CODE           	6BCC	0000	899

main_OLED.c estimated size: 899

C:\Program Files\Microchip\xc8\v1.35\sources\common\Umul16.c
		___wmul        		CODE           	66EC	0000	39

C:\Program Files\Microchip\xc8\v1.35\sources\common\Umul16.c estimated size: 39

Alteri.h
		_delay_ms      		CODE           	67BC	0000	55

Alteri.h estimated size: 55

C:\Program Files\Microchip\xc8\v1.35\sources\common\awdiv.c
		___awdiv       		CODE           	690C	0000	133

C:\Program Files\Microchip\xc8\v1.35\sources\common\awdiv.c estimated size: 133

shared
		usint2decascii@F38		MEDIUMCONST    	7783	0000	11
		_ssd1306xled_font6x8		MEDIUMCONST    	753F	0000	553
		__initialization		CODE           	66D6	0000	13
		_img0_128x64c1 		MEDIUMCONST    	778D	0000	1025
		_ssd1306xled_font8x16		MEDIUMCONST    	6F4F	0000	1521
		_img1_128x64c1 		MEDIUMCONST    	7B8D	0000	1025
		_ssd1306_init_sequence		MEDIUMCONST    	7767	0000	29

shared estimated size: 4177

ssd1306xled.c
		_ssd1306_send_byte		CODE           	67F2	0000	65
		_ssd1306_setpos		CODE           	6738	0000	41
		_ssd1306_numdecp_font6x8		CODE           	6712	0000	39
		_ssd1306_xfer_stop		CODE           	666A	0000	11
		_ssd1306_send_command_stop		CODE           	665A	0000	7
		_ssd1306_send_command_start		CODE           	6686	0000	19
		_ssd1306_char_font6x8		CODE           	6832	0000	67
		_ssd1306_send_command		CODE           	6698	0000	19
		_ssd1306_send_data_stop		CODE           	6654	0000	7
		_ssd1306_xfer_start		CODE           	6660	0000	11
		_ssd1306_send_data_start		CODE           	6674	0000	19
		_ssd1306_fill  		CODE           	66AA	0000	23
		_ssd1306_init  		CODE           	6760	0000	45
		_ssd1306_fill2 		CODE           	66C0	0000	23
		_ssd1306_fill4 		CODE           	6874	0000	71
		_ssd1306_draw_bmp		CODE           	6990	0000	151
		_ssd1306_numdec_font6x8		CODE           	678C	0000	49
		_ssd1306_string_font6x8		CODE           	68BA	0000	83

ssd1306xled.c estimated size: 750

